S123B6008E00FFBDB797BDB7BCBDB776BDB61120F8BDB71CC1FF2717C1002514C108221055
S123B6205818CEB636183A18EE0018AD0020E2398E00FF7EB609B6A4B693B630B648B6B1CC
S123B640B66CB683B676B65CBDB7423C383C183CBDB6111838180926F3183839BDB7423C0A
S123B660CE014D0926FD180926F63839BDB74218E600BDB72E39BDB742BDB73C18E700BD1F
S123B680B70A39BDB742BDB73C18EA0018E700BDB70A39BDB742BDB73C5318E40018E700DA
S123B6A0BDB70A39BDB73CBDB7ACBDB72EBDB70A39BDB73CBDB74218DF8518CE0089188FAE
S123B6C0BDB742188CFFFF270B188F18ED001808180820EA7F10201AEE008640B81020B7CA
S123B6E010203CCE1000FC100ED3851AA30E2AFBD385ED18180926F31D00403808089C873B
S123B70026D57F102038BDB70A3937C601BDB769C601BDB769C601BDB7693339E600C1FF57
S123B72027060808E6000839C6FF0808083937C600BDB769BDB76933BDB769390808E60095
S123B74008393637A60081FF270C08A60008E60008188F333239CCFFFF08080820F3F610FA
S123B7602EC42027F9F6102F3936B6102E848027F9F7102F323937CE0000BDB75EE700C1B7
S123B780FF270F08BDB75EE70008BDB75EE7000820E8CE0000333936B6102884DFB710282E
S123B7A086B0B7102B860CB7102D3239C40FF71030F61030C48027F9F6103139B610399ABF
S108B7C080B7103939C7
S105BFFEB60087
S9030000FC
